:020000040000FA
:1000000086018701831607309F000F308100093079
:1000100093009417073085008601183087008312FB
:10002000AB010230AC00BE011130BF00283094009B
:100030008822B41BF32015216400482064001B288B
:100040001F398207EB348834B334BA34D8347A3465
:100050007B34A834FB34FA34E934D9347334633450
:100060002034F134DA3400341F398207C0342034AC
:10007000A0340034803440346034E034003404343C
:1000800002340634013405340334073400340034B8
:100090000721D030FD200030FD200E210721D13076
:1000A000FD208316911583128C118C1D5528130881
:1000B000B4008316111683128C118C1D5D28130851
:1000C000B5008316111683128C118C1D6528130838
:1000D000B6008316111683128C118C1D6D2813081F
:1000E000B7008316111683128C118C1D7528130806
:1000F000B8008316111683128C118C1D7D281308ED
:10010000B9008316111683128C118C1D85281308D3
:10011000BA008316111283120E213408A000340E87
:10012000A1003508A200350EA3003608A400360E43
:10013000A500B7030319B128B7030319B728B703FC
:100140000319BE28B7030319C528B7030319CC2820
:10015000B7030319D3280D30A600A7010830A80063
:10016000D9280B30A600A7010A30A800D9280E30E4
:10017000A6000730A7000830A800D9280C30A60038
:100180000F30A7000D30A800D9280E30A600073088
:10019000A7000430A800D9280E30A6000730A70019
:1001A0000A30A800D9280630A6001030A7000D306C
:1001B000A8003808AF00380EB0003908AD00390E7D
:1001C000AE003A08A9003A0EAA000F30A005A1051A
:1001D000A205A305A405A505A905AA05AD05AE05BB
:1001E000AF05B0050800B4130721D030FD20003062
:1001F000FD203408FD200E210800831293008C118D
:100200008C1D00298316111BFD28831208008C11F8
:100210008316111483128C1D0B2908008C11831670
:10022000111583128C1D12290800C830B100B201CB
:100230000830850020303207840000082020860026
:100240003E083202031C38293F08320203183829BD
:1002500008303202031C322910303202031C3429C8
:100260008511352905163529851632083420870071
:10027000201849213C30BC00BC0B3C29B20A11308B
:100280003202031C1829B10B172985150512851296
:10029000080003110230320203190615031104305D
:1002A00032020319061503110D3032020319061527
:1002B00003110F3032020319061508000518080053
:1002C0001521051808001521051808000F30BD007C
:1002D0000930BE000D30BF002908C0002A08C10047
:1002E0006400851C5222051D5B220A30410203185E
:1002F000C1014008A9004108AA001521051C89294F
:10030000BD0B7029BA012A08BA00BA0E2908BA052D
:10031000642A0F30BD000F30BE001130BF002F081F
:10032000C0003008C1006400851C5222051D5B22FC
:10033000043041020318C1014008AF004108B00079
:100340001521051CAC29BD0B9329B8013008B80054
:10035000B80E2F08B805642A0F30BD000D30BE005E
:100360000F30BF002D08C0002E08C1006400851C9E
:100370005222051D5B22043041020318C1014008CE
:10038000AD004108AE001521051CCF29BD0BB629D3
:10039000B9012E08B900B90E2D08B905642A0F302D
:1003A000BD000630BE000930BF003708C000640041
:1003B000851C5222051D5B22083040020318C00133
:1003C0004008B70048201521051CE929BD0BD72995
:1003D000642A0F30BD000430BE000630BF00240880
:1003E000C0002508C1006400851C5222051D5B2247
:1003F000033041020318C1014008A4004108A500D0
:100400001521051C0C2ABD0BF329B6012508B600E1
:10041000B60E2408B605642A0F30BD000230BE00B7
:100420000430BF002208C0002308C1006400851CFE
:100430005222051D5B22063041020318C10140080B
:10044000A2004108A3001521051C2F2ABD0B162A66
:10045000B5012308B500B50E2208B505642A0F3092
:10046000BD000030BE000230BF002008C0002108DF
:10047000C1006400851C5222051D5B22063041022A
:100480000318C1014008A0004108A1001521051C66
:10049000642ABD0B392AB4012108B400B40E200827
:1004A000B405642A1521C00A0A3040020319C10AA2
:1004B0000F30BD0008001521C0030A3040020318A8
:1004C000C1030F30BD0008000721D030FD200030EF
:1004D000FD20B4133408FD203508FD2036133608FE
:1004E000FD203708FD203808FD203908FD203A0896
:1004F000FD200E21BE011130BF0008003613072178
:10050000D030FD200230FD203608FD200E210800ED
:100510000721D030FD200030FD200E210721D130F1
:10052000FD208C118316911583128C1D952A1308BA
:0C053000B4008316111283120E21080083
:02400E00353F3C
:00000001FF
